:100000000C9476020C9436070C9493020C94930291
:100010000C9493020C9493020C9493020C9493020C
:100020000C9493020C9493020C9493020C949302FC
:100030000C9493020C9493020C9493020C949302EC
:100040000C9493020C9493020C9493020C949302DC
:100050000C9493020C9493020C9493020C949302CC
:100060000C9493020C9493023030303030303030A6
:100070003030303030303030303030000041542BB0
:1000800043474E535057523D310D0A0041542B43C4
:10009000474E535057523D300D0A0041542B4347B1
:1000A00050535057523D300D0A0041542B43475096
:1000B000535253543D310D0A0041542B4347505382
:1000C0005253543D300D0A0041542B43475053497D
:1000D0004E463D300D0A002B434750535354415474
:1000E00055533A204C6F636174696F6E203244201F
:1000F000466978002B434750535354415455533A63
:10010000204C6F636174696F6E20334420466978B8
:100110000041542B434750535354415455533F0DC2
:100120000A0041542B434750535057523D310D0A5A
:100130000041542B4342430D0A0041542B43495084
:1001400047534D4C4F433D312C310D0A002B534149
:100150005042523A20312C310041542B53415042ED
:10016000523D302C310D0A0041542B534150425224
:100170003D322C310D0A0041542B53415042523D27
:10018000312C310D0A0041542B53415042523D3322
:100190002C312C22505744222C22696E7465726EC9
:1001A0006574220D0A0041542B53415042523D3395
:1001B0002C312C2255534552222C22696E746572C3
:1001C0006E6574220D0A0041542B53415042523D3A
:1001D000332C312C2241504E222C22696E746572D0
:1001E0006E6574220D0A0041542B53415042523D1A
:1001F000332C312C22434F4E54595045222C224748
:10020000505253220D0A000A424154544552595B40
:100210006D565D3D00204C415449545544453D00C8
:10022000204C4F4E475449545544453D000D0A005B
:100230002C000D0A20687474703A2F2F6D61707352
:100240002E676F6F676C652E636F6D2F6D617073B6
:100250003F713D0041542B434E45544C494748544F
:100260003D300D0A00415426570D0A0041542B49D8
:1002700050523D393630300D0A0041542B43534320
:100280004C4B3D300D0A0041542B4353434C4B3DE6
:10029000310D0A0041542B4346554E3D310D0A00A5
:1002A00041542B4346554E3D340D0A0041542B43D7
:1002B0004C49503D310D0A00220A0D00475541526C
:1002C00044204D4F44452053544F50504544004125
:1002D0004C4552542C20504F534954494F4E2043C3
:1002E00048414E47454420544F203A20200047556E
:1002F000415244204D4F44452041435449564154B6
:1003000045442E2E20504C454153452057414954D9
:100310002035204D494E55544553204245464F52B5
:1003200045204E45585420434F4D4D414E440A0000
:100330004143544956415445442043414C4C532079
:1003400046524F4D20004D554C5449504C45204D80
:100350004541535552454D454E545320494E20502A
:10036000524F47524553532E2E20504C4541534532
:100370002057414954203235204D494E555445535C
:10038000204245464F5245204E45585420434F4D3C
:100390004D414E440A0053494E474C45204D45417E
:1003A000535552454D454E5420494E2050524F47CB
:1003B000524553532E2E2E20504C45415345205725
:1003C00041495420372D38204D494E55544553202E
:1003D0004245464F5245204E45585420434F4D4DBF
:1003E000414E440A00434F4D4D414E44204143434A
:1003F00045505445440A0053544F5000475541520C
:10040000440041435449564154450053494E474CDA
:1004100045004D554C544900434D543A0041542B2E
:10042000434E4D493D312C322C302C302C300D0AAE
:100430000041542B434D4744413D2244454C20410B
:100440004C4C220D0A0041542B434D47533D220092
:1004500041542B434D47463D310D0A004154480A53
:100460000D0041542B43464752493D310A0D00418E
:10047000542B4350494E3D2231313131220A0D0077
:10048000415445300A0D0041542B4350494E3F0A18
:100490000D002B4350494E3A2053494D2050494EB0
:1004A000002B4350494E3A20524541445900415493
:1004B0002B435245473D300A0D0041542B435245D2
:1004C000473F0A0D002B435245473A20302C350058
:1004D0002B435245473A20302C310052494E4700B9
:1004E0004F4B0041540041540A0D000011241FBE1F
:1004F000CFEFD8E0DEBFCDBF13E0A0E0B1E0E6E78C
:10050000FEE102C005900D92A231B107D9F713E0C8
:10051000A2E1B3E001C01D92A334B107E1F70E944C
:1005200041070C94390F0C94000082E08093C000C6
:100530001092C5008CE08093C400E1ECF0E0808173
:1005400088608083808180618083E2ECF0E080813C
:100550008660808308959091C00095FFFCCF8093C2
:10056000C60008958091C00087FFFCCF8091C6002F
:100570000895EF92FF920F931F93CF93DF939C0107
:10058000182FFC0190E08E2F811B841748F5A19154
:10059000EB01C90FD11D5881A513F5CF90E0592F5C
:1005A000580FD901A50FB11D0C91C92FD0E0011131
:1005B0000CC0DB010D900020E9F71197A61BB70BCB
:1005C000CA17DB0701F781E00CC07B01EC0EFD1EB2
:1005D000D7015C91552369F30513EBCF9F5FDFCF04
:1005E00080E0DF91CF911F910F91FF90EF900895E0
:1005F000CF93DF93EC018991882319F00E94AB021D
:10060000FACFDF91CF910895CF93DF93EC01CE0124
:10061000FE012491222331F02196FC0184910E9455
:10062000AB02F5CFDF91CF910895CF9310924203A3
:10063000C6E90E94B202282F30E02A30310579F055
:100640002D30310561F0E0914203F0E0E859FD4FB3
:100650008083809142038F5F809342030DC080911D
:100660004203882349F0E0914203F0E0E859FD4F4E
:1006700010821092420302C0C150D9F681E0CF919E
:100680000895CF9310923F03C6E90E94B202282F2B
:1006900030E02A30310579F02D30310561F0E091FC
:1006A0003F03F0E0EA56FE4F808380913F038F5F67
:1006B00080933F030DC080913F03882349F0E09170
:1006C0003F03F0E0EA56FE4F108210923F0302C053
:1006D000C150D9F681E0CF910895CF9310923D0398
:1006E00010923E0310924203C0E00E94B202CF5F1C
:1006F0008C3219F0C431C9F75EC0C43109F45BC053
:100700000E94B202E0913D03F0E0E259FE4F808387
:1007100090913D039F5F90933D03CF5F8C3249F4EE
:10072000E0913D03F0E0E359FE4F108210923D034B
:1007300005C0C63429F7F4CFC63480F40E94B20253
:10074000E0913E03F0E0EE57FE4F808390913E0330
:100750009F5F90933E03CF5F8C3271F7E0913E0331
:10076000F0E0EF57FE4F108210923E0305C02A3092
:100770003105A9F0C63498F40E94B202282F30E067
:10078000E0914203F0E0E859FD4F808380914203FD
:100790008F5F80934203CF5F2D30310541F7E091A9
:1007A0004203F0E0E959FD4F1082109242030E948B
:1007B000B20281E001C080E0CF910895CF93109202
:1007C0004103C0E00E94B202CF5F8A3311F0C63904
:1007D000C9F70E94B202CF5F823211F0C639C8F366
:1007E0000E94B202E0914103F0E0EC5AFD4F808399
:1007F000909141039F5F90934103CF5F823249F410
:10080000E0914103F0E0ED5AFD4F10821092410358
:1008100007C0C63928F3F4CF0D9749F0C63938F42C
:100820000E94B20290E0CF5F8A309105A9F781E083
:10083000CF910895109241031092420380E0E0911D
:100840004203F0E0E859FD4F2081909142039F5F01
:10085000909342038F5F2A3311F0863981F7E0913C
:100860004203F0E0E859FD4F2081909142039F5FE1
:10087000909342038F5F223211F0863980F3E0912A
:100880004203F0E0E859FD4F2081909142039F5FC1
:1008900090934203E0914103F0E0EC5AFD4F208336
:1008A000909141039F5F909341038F5F223211F03B
:1008B000863928F3E0914103F0E0ED5AFD4F1082B4
:1008C000109241031092420381E00895CF93109259
:1008D0001303C0E00E94B202CF5F8C3219F0C6341D
:1008E000C9F72BC0C63449F10E94B202CF5F8C32E7
:1008F00011F0C634C9F70E94B202282F30E0E0910F
:100900001303F0E0E050FF4F8083809113038F5F6B
:1009100080931303CF5F2A30310529F02D30310544
:1009200011F0C63440F3E0911303F0E0E150FF4FC3
:1009300010821092130381E001C080E0CF910895EE
:10094000CF9310923D0310923E0310923C0388EC2B
:1009500090E00E940403C0E00E94B202CF5F8A339D
:1009600019F0C431C9F775C0C43109F472C00E94CE
:10097000B202CF5F8C3211F0C639C9F70E94B202C1
:10098000E0913E03F0E0EE57FE4F808390913E03EE
:100990009F5F90933E03CF5F8C3249F4E0913E031A
:1009A000F0E0EF57FE4F108210923E0305C0C639AB
:1009B00028F3F4CFC63980F40E94B202E0913D03DF
:1009C000F0E0E259FE4F808390913D039F5F90934A
:1009D0003D03CF5F8C3271F7E0913D03F0E0E359C6
:1009E000FE4F108210923D0302C0C63940F40E94AF
:1009F000B202CF5F8C32C9F702C0C63940F40E9400
:100A0000B202CF5F8C32C9F702C0C63940F40E94EF
:100A1000B202CF5F8C32C9F702C0C63980F40E949F
:100A2000B202E0913C03F0E0E65FFE4F80839091DC
:100A30003C039F5F90933C03CF5F8C3271F7E09152
:100A40003C03F0E0E75FFE4F108210923C0381E030
:100A500001C080E0CF910895882361F026E033E162
:100A60004EEA4A95F1F73A95E1F72A95D1F700C099
:100A70008150F2CF0895CF93DF938091120381309C
:100A800021F0809112038530C9F481E090E00E944A
:100A90002C058DE790E00E94040382E090E00E9424
:100AA0002C0582E291E00E94040382E090E00E9423
:100AB0002C0589EB90E00E94040304C081E090E0E3
:100AC0000E942C05C0E0809112038F3F21F08FE03F
:100AD00090E00E942C0581E191E00E9404030E94B5
:100AE0001503882309F448C04DE150E064EF70E03D
:100AF00084E193E00E94F60E4AEA64E173E088E63E
:100B000092E00E94B902D82FC33119F0D13099F484
:100B100018C04DE150E067ED70E084E193E00E9481
:100B2000F60E4AEA64E173E088E692E00E94B902B8
:100B3000813061F706C0809112038F3FC1F1CF5F12
:100B40001BC00E94A00482E090E00E942C05C0918E
:100B50001203C13071F58BE990E00E94040381E03B
:100B600090E00E942C058CE890E00E94040381E054
:100B700090E00E942C051EC0C43108F4A4CF82E08E
:100B800090E00E942C0580911203813081F48BE962
:100B900090E00E94040381E090E00E942C058CE824
:100BA00090E00E94040381E090E00E942C05C0E0E8
:100BB00001C0C1E08C2FDF91CF91089520E12A95EB
:100BC000F1F700C00895CF9386EE94E00E940403ED
:100BD0000E94150343E050E0882319F060EE74E0B2
:100BE00002C063EE74E084E193E00E94F60E4AEAEC
:100BF00064E173E088E692E00E94B902C1E08130CE
:100C000009F0C0E081E00E942C05CC23E9F281E0EC
:100C10000E942C0580E894E00E94040381E00E9479
:100C20002C0581E0CF910895CF9382E00E942C059E
:100C300087E894E00E9404030E9415038823A9F327
:100C40004DE050E061EA74E084E193E00E94F60E2A
:100C50004AEA64E173E088E692E00E94B902C82F94
:100C60004FE050E062E974E084E193E00E94F60E08
:100C70004AEA64E173E088E692E00E94B9028130BA
:100C800049F40E942C058FE694E00E94040381E061
:100C90000E942C05C13049F681E0CF910895CF9391
:100CA000DF9381E00E942C058AEB94E00E9404030C
:100CB0000E941503811109C081E00E942C0584E97E
:100CC00092E00E940403C8E124C04BE050E060EDD4
:100CD00074E084E193E00E94F60E4AEA64E173E076
:100CE00088E692E00E94B902813009F47CC04BE0B2
:100CF00050E065EC74E084E193E00E94F60E4AEA6D
:100D000064E173E088E692E00E94B9028130A1F6C6
:100D10006AC088E70E942C058AEB94E00E940403D5
:100D20000E941503882309F460C04BE050E060ED99
:100D300074E084E193E00E94F60E4AEA64E173E015
:100D400088E692E00E94B902D82F4BE050E065ECB3
:100D500074E084E193E00E94F60E4AEA64E173E0F5
:100D600088E692E00E94B9028130E9F181E0D13059
:100D700009F43FC00E942C0580EA92E00E9404031F
:100D800081E00E942C058CE890E00E94040381E041
:100D90000E942C058BE990E00E94040381E00E94F0
:100DA0002C0587E892E00E940403DEE18CE30E94B8
:100DB0002C05D150D9F7459886EE94E00E940403A3
:100DC00081E00E942C058AE792E00E94040381E002
:100DD0000E942C05459A81E00E942C0584E992E04E
:100DE0000E94040302C081E004C0C15009F091CF09
:100DF00080E0DF91CF91089581E00E942C0587EE7D
:100E000091E00E94040381E00E942C0587EC91E0B0
:100E10000E94040381E00E942C0586EA91E00E9472
:100E2000040381E00E942C0586E891E00E940403FF
:100E300081E00E942C0581E0089583B7817F846062
:100E400083BF83B7816083BF52985A9AF894E9E6CA
:100E5000F0E080818D7F808380818E7F8083E89A1F
:100E60007894889583B78E7F83BF08951F920F92E1
:100E70000FB60F921124E8980F900FBE0F901F909D
:100E800018951092120352985A9A3D9A459A45E144
:100E900050E068E670E082E391E00E94F60E45E1E2
:100EA00050E068E670E08AE591E00E94F60E45E1C8
:100EB00050E068E670E08EE191E00E94F60E45E1B8
:100EC00050E068E670E086E491E00E94F60E0E9431
:100ED00095028AE00E942C0580E894E00E940403B9
:100EE00081E00E942C050E94E30581E00E942C0510
:100EF0008CE692E00E94040381E00E942C0584E9C4
:100F000092E00E94040381E00E942C058EEA94E0A6
:100F10000E94040381E00E942C0585E692E00E9475
:100F2000040383E00E942C050E94140681E00E94C5
:100F30002C0580E594E00E94040381E00E942C05CA
:100F400081E394E00E9404038AE50E942C050E943C
:100F50004F0620EA822E26E8922EAA24A394B12CD2
:100F6000DFEF15E01092120381E00E942C058CEA5D
:100F700092E00E94040381E00E942C0580E594E049
:100F80000E94040381E00E942C058DE194E00E9400
:100F9000040381E00E942C058CE890E00E94040389
:100FA00081E00E942C058BE990E00E94040381E01F
:100FB0000E942C0587E892E00E94040382E00E94D0
:100FC0002C058091C00087FF03C08091C600F9CF37
:100FD00090E8C92E98EAD92E92E1E92EFF24F394E5
:100FE0008091C00087FD30C00E94DE0581E0C81AF4
:100FF000D108E108F108A1F7459886EE94E00E9437
:10100000040381E00E942C058AE792E00E94040319
:1010100081E00E942C05459A81E00E942C050E94E7
:101020004F0681E00E942C0587E892E00E940403AD
:1010300081E00E942C05109212038091C00087FF6E
:10104000C7CF8091C600F9CF0E941503882309F409
:101050002CC245E050E068E174E084E193E00E9436
:10106000F60E4AEA64E173E088E692E00E94B90273
:10107000813009F08EC10E9441030E941A0410922F
:10108000120346E050E062E174E084E193E00E94E4
:10109000F60E86E991E00E94FF0E4AEA64E173E0F1
:1010A0000E94B902813009F045C0459886EE94E06F
:1010B0000E94040381E00E942C058AE792E00E94CE
:1010C000040381E00E942C05459A81E00E942C05D2
:1010D00080E594E00E94040381E00E942C0586E4F0
:1010E00094E00E94040384E592E00E94F80288EBF9
:1010F00092E00E94040381E00E942C0586E493E0C4
:101100000E9404038AE10E94AB028AE00E942C053F
:1011100080E594E00E94040381E00E942C0581E3B5
:1011200094E00E94040382E00E942C0510931203B5
:10113000C1E001C0C0E047E050E06BE074E084E152
:1011400093E00E94F60E86E991E00E94FF0E4AEAC3
:1011500064E173E00E94B902082F813009F044C0B5
:10116000459886EE94E00E94040381E00E942C05DD
:101170008AE792E00E94040381E00E942C05459AD0
:1011800081E00E942C0580E594E00E94040381E048
:101190000E942C0586E494E00E94040384E592E01A
:1011A0000E94F80288EB92E00E94040381E00E9412
:1011B0002C0586E993E00E9404038AE10E94AB02B9
:1011C0008AE00E942C0580E594E00E94040381E0FF
:1011D0000E942C0581E394E00E94040382E00E94B7
:1011E0002C0500931203C1E049E050E062E074E096
:1011F00084E193E00E94F60E86E991E00E94FF0EE2
:101200004AEA64E173E00E94B902813009F052C0F9
:10121000459886EE94E00E94040381E00E942C052C
:101220008AE792E00E94040381E00E942C05459A1F
:1012300081E00E942C0544E150E060E070E084E52C
:1012400092E00E94210F80E594E00E94040381E077
:101250000E942C0586E494E00E94040384E592E059
:101260000E94F80288EB92E00E94040381E00E9451
:101270002C0580E393E00E94040384E592E00E9441
:10128000F8028AE10E94AB028AE00E942C0580E508
:1012900094E00E94040381E00E942C0581E394E025
:1012A0000E94040382E00E942C051092120301E0C8
:1012B000C0E001C00C2F46E050E06CEF73E084E129
:1012C00093E00E94F60E86E991E00E94FF0E4AEA42
:1012D00064E173E00E94B902813009F05CC0459876
:1012E00086EE94E00E94040381E00E942C058AE7C8
:1012F00092E00E94040381E00E942C05459A81E05F
:101300000E942C0580E594E00E94040381E00E9485
:101310002C0586E494E00E94040384E592E00E9498
:10132000F80288EB92E00E94040381E00E942C0501
:101330008EEE92E00E9404038AE10E94AB028AE0F2
:101340000E942C0580E594E00E94040381E00E9445
:101350002C0581E394E00E94040382E00E942C05A6
:10136000D09312038DE790E00E94040382E00E9474
:101370002C0582E291E00E94040382E00E942C0589
:1013800089EB90E00E94040381E00E942C0501E0BB
:1013900001C000E0C1E045E050E06BED74E084E1A5
:1013A00093E00E94F60E4AEA64E173E088E692E078
:1013B0000E94B902813009F041C045980E94DE03C5
:1013C00086EE94E00E94040381E00E942C058AE7E7
:1013D00092E00E94040381E00E942C05459A81E07E
:1013E0000E942C058CE594E00E94040381E00E9499
:1013F0002C0580E594E00E94040381E00E942C0506
:1014000081E394E00E94040382E00E942C0544E101
:1014100050E060E070E080E492E00E94110F44E14F
:1014200064E572E080E492E00E94B902813019F430
:10143000809312033AC01092120302C0011132C00D
:10144000459886EE94E00E94040381E00E942C05FA
:101450008AE792E00E94040381E00E942C05459AED
:1014600081E00E942C050E9414060E944F0681E034
:101470000E942C0580E594E00E94040381E00E9414
:101480002C0581E394E00E94040382E00E942C0575
:1014900089E591E00E94040385E00E942C051092EA
:1014A000120360CDCC2309F45DCD0E943B05813051
:1014B00009F003C2CEE6D1E009900020E9F72197B8
:1014C000CE56D140DD27FE01E459FE4FC080D12C1D
:1014D00090E3C91AD108EE24D7FCE094FE2CFE015B
:1014E000E559FE4FA081B0E0D097FE01E659FE4FCE
:1014F000408150E0405351092AE030E00E948D0EB7
:101500002B013C0124E630E0DA010E948D0E460EEC
:10151000571E681E791EC40CD51CE61CF71CFE0164
:10152000E759FE4FA081B0E0D09728EE33E00E944B
:101530008D0EC60ED71EE81EF91EFE01E859FE4F9D
:10154000A081B0E0D09720E137E20E948D0EC60E58
:10155000D71EE81EF91EFE01EA59FE4FA081B0E039
:10156000D09720EA36E841E050E00E94940EC60E83
:10157000D71EE81EF91EFE01EB59FE4FA081B0E018
:10158000D09720E432E44FE050E00E94940E6C0DBE
:101590007D1D8E1D9F1D2CE330E040E050E00E9439
:1015A0009C0E29013A01FE01EC59FE4FA081B0E0EA
:1015B000D09720E836E948E950E00E94940E6B018C
:1015C0007C01CB30D10540F1FE01ED59FE4F808109
:1015D0008D3269F0A081B0E0D09720E031EE45EF88
:1015E00055E00E94940EC60ED71EE81EF91ECC30A0
:1015F000D10590F0CE59DE4F88818D3269F0A881F7
:10160000B0E0D09720E03AEC4AE95BE30E94940E08
:10161000C60ED71EE81EF91EC701B601640D751D62
:10162000861D971D20916E012D3209F020E3209335
:10163000460120E03AEC4AE95BE30E949C0E205D03
:101640002093470120E031EE45EF55E00E949C0ECB
:10165000205D2093480120E836E948E950E00E94E7
:101660009C0E205D209349012EE220934A0120E444
:1016700032E44FE050E00E949C0EA50194010E94CC
:101680009C0E20E137E240E050E00E949C0E205D7D
:1016900020934B0128EE33E040E050E00E949C0E86
:1016A000205D20934C0124E630E040E050E00E94B1
:1016B0009C0E205D20934D012AE030E040E050E098
:1016C0000E949C0E205D20934E01605D60934F014F
:1016D00010925001C2E8D1E009900020E9F721976B
:1016E000C258D140DD27FE01E058FE4FC080D12C0A
:1016F00080E3C81AD108EE24D7FCE094FE2CFE014A
:10170000E158FE4FA081B0E0D097FE01E258FE4FB5
:10171000408150E0405351092AE030E00E948D0E94
:101720002B013C0124E630E0DA010E948D0E460ECA
:10173000571E681E791EC40CD51CE61CF71CFE0142
:10174000E358FE4FA081B0E0D09728EE33E00E942E
:101750008D0EC60ED71EE81EF91EFE01E458FE4F80
:10176000A081B0E0D09720E137E20E948D0EC60E36
:10177000D71EE81EF91EFE01E658FE4FA081B0E01C
:10178000D09720EA36E841E050E00E94940EC60E61
:10179000D71EE81EF91EFE01E758FE4FA081B0E0FB
:1017A000D09720E432E44FE050E00E94940E6C0D9C
:1017B0007D1D8E1D9F1D2CE330E040E050E00E9417
:1017C0009C0E69017A01FE01E858FE4FA081B0E04D
:1017D000D09720E836E948E950E00E94940E2B01AA
:1017E0003C01CB30D10590F0C958DE4F88818D3255
:1017F00069F0A881B0E0D09720E031EE45EF55E0E8
:101800000E94940E460E571E681E791EC301B20137
:101810006C0D7D1D8E1D9F1D209182012D3209F0C2
:1018200020E320935A0120E031EE45EF55E00E947D
:101830009C0E205D20935B0120E836E948E950E0EA
:101840000E949C0E205D20935C012EE220935D019E
:1018500020E432E44FE050E00E949C0EA501940188
:101860000E949C0E20E137E240E050E00E949C0E76
:10187000205D20935E0128EE33E040E050E00E94BE
:101880009C0E205D20935F0124E630E040E050E0B4
:101890000E949C0E205D209360012AE030E040E031
:1018A00050E00E949C0E205D20936101605D60937A
:1018B000620110926301C1E057C0809112038F3F13
:1018C00009F4C9C0C3E081E00E942C0589E591E0DC
:1018D0000E94040384E00E942C050E94FC0687E716
:1018E00091E00E9404038AE00E942C0588E691E0C2
:1018F0000E9404030E941503882309F40CC24CE0E3
:1019000050E06DE471E084E193E00E94F60E4AEA53
:1019100064E173E088E692E00E94B90291E08130D0
:1019200009F0F9C1C15009F493C0992361F281E033
:101930000E942C058AE391E00E9404030E946D033B
:10194000C82F811103C087E30E942C0585E00E9407
:101950002C0589E591E00E94040385E00E942C0596
:10196000C13009F078C0C0E0809112038F3F09F4C4
:1019700073C081E00E942C0581E391E00E94040382
:101980000E94660481E00E942C0580E594E00E949C
:10199000040381E00E942C0586E494E00E94040385
:1019A00084E592E00E94F80288EB92E00E94040332
:1019B00081E00E942C05C11104C088E692E00E94DB
:1019C000F80280E292E00E940403C11103C08EE697
:1019D00091E002C086E491E00E94F80285E192E085
:1019E0000E940403C11103C082E891E002C08AE5AD
:1019F00091E00E94F80287E092E00E94040380E0F8
:101A000091E00E94F80282E392E00E940403C11177
:101A100003C082E891E002C08AE591E00E94F802EA
:101A200080E392E00E940403C11103C08EE691E0BE
:101A300002C086E491E00E94F8028DE292E00E94EA
:101A4000040381E00E942C058AE10E94AB0204C0DD
:101A5000913009F46CCFC0E086E391E00E94D80E8B
:101A60008C0183E291E00E94D80EC13009F08DC054
:101A7000209112032F3F09F088C0012B09F485C083
:101A8000892B09F482C086E391E00E94D80EEC0114
:101A90008EE591E00E94D80E6C0183E291E00E94F5
:101AA000D80E7C018BE491E00E94D80EE81AF90A66
:101AB000F7FE03C0F194E194F1089BEFE916F104FD
:101AC0005CF4CC19DD09D7FF03C0D195C195D109CC
:101AD000CB3FD1050CF459C081E00E942C0580E574
:101AE00094E00E94040381E00E942C0586E494E0C7
:101AF0000E94040384E592E00E94F80288EB92E0E1
:101B00000E94040381E00E942C058FEC92E00E9469
:101B1000040382E392E00E9404038AE591E00E94BC
:101B2000F80280E392E00E94040386E491E00E94C0
:101B3000F8028DE292E00E94040381E00E942C05ED
:101B40008AE10E94AB028AE00E942C0581E080932A
:101B500012038BE990E00E94040381E00E942C05AF
:101B60008CE890E00E94040381E00E942C0580E54F
:101B700094E00E94040381E00E942C0581E394E03C
:101B80000E94040382E00E942C058AE0EAE5F1E06D
:101B9000A2E3B1E001900D928A95E1F78BE0E6E4D3
:101BA000F1E0AEE1B1E001900D928A95E1F780910C
:101BB00012038F3F29F0809112038150809312030A
:101BC00080911203882369F0809112038F3F49F0BE
:101BD0008CE30E942C058CE30E942C058CE30E9470
:101BE0002C0580911203811103C08AE00E942C050C
:101BF000809112038F3F09F089C081E00E942C057B
:101C00008091C00087FF03C08091C600F9CFC12C2E
:101C100085E3D82E8CE0E82EF12C0E94DE05809121
:101C2000C00091E0C91AD108E108F10809F46EC0BA
:101C300087FFF3CF0E941503882309F467C045E0AE
:101C400050E068E174E084E193E00E94F60E4AEA15
:101C500064E173E088E692E00E94B902813009F005
:101C600055C00E9441030E941A0445E050E067EF0E
:101C700073E084E193E00E94F60E86E991E00E9411
:101C8000FF0E4AEA64E173E00E94B9028130F1F587
:101C900080E594E00E94040381E00E942C0586E424
:101CA00094E00E94040384E592E00E94F80288EB2D
:101CB00092E00E94040381E00E942C058CEB92E0EC
:101CC0000E9404038AE10E94AB028AE00E942C0574
:101CD00080E594E00E94040381E00E942C0581E3EA
:101CE00094E00E94040382E00E942C058BE990E0BE
:101CF0000E94040381E00E942C058CE890E00E9481
:101D0000040381E00E942C051092120380911203BB
:101D10008111CBCB25C990E005CE0E94BE0EB7FF46
:101D20000895821B930B0895B7FF0C94CD0E0E946B
:101D3000CD0E821B930B0895A1E21A2EAA1BBB1B8A
:101D4000FD010DC0AA1FBB1FEE1FFF1FA217B30787
:101D5000E407F50720F0A21BB30BE40BF50B661F9D
:101D6000771F881F991F1A9469F760957095809561
:101D700090959B01AC01BD01CF010895A29FB001D8
:101D8000B39FC001A39F700D811D1124911DB29FAF
:101D9000700D811D1124911D08950E94BE0EA59FF6
:101DA000900DB49F900DA49F800D911D1124089556
:101DB000FC0188279927E89421912032E9F3293002
:101DC00010F02E30C8F32B3241F02D3239F46894E4
:101DD00004C00E94090F820F911D219120532A30C7
:101DE000C0F31EF4909581959F4F0895FB01DC018F
:101DF00002C005900D9241505040D8F70895DC0183
:101E00006C9161566A3108F0605E6F5B6D93C1F74B
:101E100008957AE0979F902D879F802D910D112432
:101E20000895DC01CB01FC01F999FECF06C0F2BD9B
:101E3000E1BDF89A319600B40D9241505040B8F788
:101E40000895DC01CB0103C02D910E942C0F41505D
:101E50005040D0F70895262FF999FECF1FBA92BDB2
:101E600081BD20BD0FB6F894FA9AF99A0FBE01967B
:061E70000895F894FFCF75
:101E7600303030303030303030303030303030305C
:101E8600303030303030303030303030303030304C
:101E9600303030303030303030303030303030303C
:101EA600303030303030303030303030303030302C
:101EB600303030303030303030303030303030301C
:101EC600303030303030303030303030303030300C
:101ED60030303030303030303030303030303030FC
:101EE60030303030303030303030303030303030EC
:101EF60030303030303030303030303030303030DC
:101F0600303030303030313233343536373839309E
:101F16003132333435363738393031323334353679
:101F26003738393031323334353637383930313263
:101F3600333435363738393031323334353637384D
:101F4600393031323334353637383930313233344B
:101F5600353637383930313233343536373839302B
:101F66003132333435363738393031323334353629
:101F76003738393031323334353637383930313213
:101F860033343536373839303132333435363738FD
:101F960039303132333435363738393031323334FB
:101FA60035363738393031323334353637383930DB
:101FB60031323334353637383930313233343536D9
:101FC60037383930313233343536373839303132C3
:101FD60033343536373839303132333435363738AD
:101FE60039303132333435363738393031323334AB
:101FF600353637383930313233343536373839308B
:102006003132333435363738393031323334353688
:102016003738393031323334353637383930313272
:10202600333435363738393031323334353637385C
:10203600393031323334353637383930313233345A
:10204600353637383930313233343536373839303A
:102056003132333435363738393031323334353638
:102066003738393031323334353637383930313222
:10207600333435363738393031323334353637380C
:022086003930EF
:00000001FF
